:030000000212AF3A
:03000B000200C12F
:03002B000203EBE2
:03005B000205B8E3
:030073000205AED5
:1000800002030406080C10182030406080020304AC
:1000900006080C101820304080FF0406080C1018C9
:1000A0002030406080A0C000000001010003020277
:1000B000010D0D040206020D0505050D06030502DE
:1000C00002C2AFC0D0C0E0205A0D302F02E473301E
:1000D000600280F90203D7306306C2B1C287C281D1
:1000E00085258AC25AE525F4700221CA056130606F
:1000F00013206A19758B00D0E0D0D0C2B1C287C27C
:1001000081D2AF32C2B1C287C2810201BAD26EC2FD
:100110006FE565601CC3E5611495654014C26ED23D
:100120006FC3E561956450030201BA756100020175
:10013000BA206C14C2B1C287C2817406D5E0FDD268
:1001400082D286D2800201BAD26FC2B1C287C28186
:10015000E53D20E23420E1127406D5E0FD20750271
:10016000D280307502D2820201BA20E0127406D524
:10017000E0FD207502D280307502D2820201BA748D
:1001800006D5E0FDD2860201BA20E11F20E00A7404
:1001900006D5E0FDD2860201BA7406D5E0FD2075D1
:1001A00002D282307502D2800201BA7406D5E0FD17
:1001B000207502D282307502D280758B00D0E0D0DB
:1001C000D0C2B1C287C281D2AF32D0E0D0D0D2AFDC
:1001D0003261D7E525600A207502D2B1307502D2AE
:1001E00081C28761D7E5256002D287207502C2816E
:1001F000307502C2B161D7E525600A207502D2814F
:10020000307502D2B1207502C2B1307502C281616F
:10021000D7207502C282307502C280E525600A20AF
:100220007502D2B1307502D281207502C28030755C
:1002300002C282C28761D7207502C282307502C2B3
:1002400080207502C280307502C2827406D5E0FD3E
:10025000E525600A207502D2B1307502D281C287CD
:1002600061D7207502C282307502C280E525600A1E
:10027000207502D2B1307502D281C286C28761D7A1
:10028000207502C282307502C280C2867406D5E033
:10029000FDE525600A207502D2B1307502D281C217
:1002A0008761D7C286E5256002D287207502C282A7
:1002B000307502C280207502C281307502C2B16100
:1002C000D7C286207502C282307502C2807406D5FC
:1002D000E0FDE5256002D287207502C281307502FB
:1002E000C2B161D7C286E5256002D287207502C2FD
:1002F00080307502C282207502C281307502C2B19F
:1003000061D7C286207502C280307502C28274062F
:10031000D5E0FDE5256002D287207502C2813075E7
:1003200002C2B161D7207502C280307502C282E577
:1003300025600A207502D281307502D2B1C28620B2
:100340007502C2B1307502C28161D7207502C280C8
:10035000307502C282C2867406D5E0FDE525600ACA
:10036000207502D281307502D2B1207502C2B1303F
:100370007502C28161D7207502C280307502C282C7
:10038000E525600A207502D281307502D2B1207550
:1003900002C282307502C280207502C2B13075027D
:1003A000C28161D7207502C280307502C282207579
:1003B00002C282307502C2807406D5E0FDE5256078
:1003C0000A207502D281307502D2B1207502C2B105
:1003D000307502C28161D7E525F4F58A758B007509
:1003E0006000D25AD0E0D0D0D2AF32C2AFC0D0C0BD
:1003F000E0D2D3C2CEE528600A741F552E6049159D
:1004000028814878007900E580307601F430E502F3
:1004100078FF53DACF20760343DA2030760343DACD
:1004200010C2D8C269E580307601F430E50279FF68
:10043000C3E89970CE305903752840741F552E605B
:10044000037528408858D268E52960041529815B26
:10045000741F552E600543DA01C2D820680281E07E
:10046000E558F8C268741F552E60367982B704319A
:0F047000C3E894F0400374F0F8E8C4540F28F880
:10047F007984B7030281A1C313C313872120080214
:10048F00C313200A06C3C898F881A128F850037433
:10049F00FFF8C3E8955F5003E55FF8E52C5406704D
:1004AF0030882230630AC3E522955C4003855C22C5
:1004BF007882B6041CC3E5229524401278A096409A
:1004CF000DE52426F52450097524FF0204E085224A
:1004DF002420CF09D0E0D0D0C2D3D2AF32C2CF7850
:1004EF0001E5286008741F552E70021528C3E558C2
:1004FF0094014005755B00A10FE55B046002055B8D
:10050F007982B7020EE548601EC3E5229432401788
:10051F008547227982B7030FE548600BC3E5229424
:10052F00324004798E8722C3E52395226008400468
:10053F001523A1450523D8C80562E562700215622F
:10054F00D563537563017803C3E562941E4047C3B7
:10055F00E562946450087801756303020579C3E579
:10056F0062949650057801756301C3E55D9524404B
:10057F0018E548701485245DE56204600375621EFA
:10058F0075630175233C0205A5C3E55D285005750C
:10059F005DFFA1A5F55DD0E0D0D0C2D3D2AF32C2FE
:1005AF00AF53917FC258D2AF32C2AFC0D0C0E0C0FC
:1005BF00F0D2D3A8FBA9FCC2D8306902C11B53DA11
:1005CF00CF20760343DA1030760343DA20D269E581
:1005DF0080307601F420E502A1EF88268927E1BB60
:1005EF0053DACF20760343DA2030760343DA10C292
:1005FF00D8C269741F552E7002E1A17800E58030D2
:10060F007601F430E502E1A18858E1A153DACF2059
:10061F00760343DA2030760343DA10C26920590299
:10062F00C1D553DACF20760343DA1030760343DA9D
:10063F0020C2D8D26988538954C3E89551F8E995F7
:10064F0052F9E4FB7AFAC3E894C8E994005008E43D
:10065F00D2E4FB7A0AC1A8C3E89468E99401500870
:10066F00E4D2E3FB7A0FC1A8C3E894D0E994025017
:10067F0008E4D2E2FB7A1EC1A8C3E894A0E994056E
:10068F005008E4D2E1FB7A3CC1A8C3E89498E994FE
:10069F00085006E4D2E0FB7A78C3E89555FCE9955B
:1006AF0056FD30E708ECF42401FCEDF4FD7557001E
:1006BF007008C3EC9A500375570188558956A85393
:1006CF00A95488518952C3E89526F8E99527F9303E
:1006DF007402E174307302E174307202E16DE9C3A8
:1006EF0013F9E813F8307102E16DE9C313F9E81358
:1006FF00F8307002E16DE9C313FDE813FC205918BF
:10070F00C3EC941CED940240030207A1ED7009C3E2
:10071F00EC94C850030207BB74002077037896E669
:10072F0024FAFEE43400FFC3EC9EFCED9FFD50065F
:10073F0078007900E174C3EC94FFED9400400678E3
:10074F00FF7900E174EC856CF0A4C5F0A2F733F8E3
:10075F007900400302079078FF7900020790E9C300
:10076F0013F9E813F830740EE9600278FFC3E81349
:10077F0038F8E43400F9C3E894FFE99400400278B4
:10078F00FF8858D268205902E1A1741FF4552E4BEF
:10079F00F52E752840741F552E700375280A305991
:1007AF0002E1BB741F552E600353DAFE75292074C6
:1007BF001F552E700375290AD0F0D0E0D0D0C2D3C8
:1007CF00D2AF327901E1EA7903E1EA790AE1EA7914
:1007DF001EE1EA7964E1EA79C8E1EA7817E4D5E045
:1007EF00FDD8FAD9F6227A147B780208117A107B99
:1007FF008C0208117A0D7BB40208117A0B7BC802A8
:10080F000811AC257525017902B275E4C286D5E0D1
:10081F00FDE5256002D287D5E0FDC287D5E0FDD288
:10082F0086D5E0FDE525600A207502D2B13075024C
:10083F00D281E56DD5E0FD207502C2B1307502C2DF
:10084F00817496D5E0FDD9C1EAF8D5E0FDD8FBDB80
:10085F00B1C2868C2522C37C007D0075F00005F0A7
:0F086F00EA33FAEB33FB50F6EB13FBEA13FAC351
:10087E00E9FFE8FEE89AF8E99BF95004EFF9EEF883
:10088E00B3EC33FCED33FDD5F0DFEDF9ECF822E8F7
:10089E0089F08A20D2D4F8A9F07B0030F70B7BFFC9
:1008AE00F42401F8E9F43400F9E88520F0A4ADF061
:1008BE00F8E98520F0A4AFF0FEED2EF974003FFAB2
:1008CE007C04C3EA13FAE913F9E813F8DCF48BF0AD
:1008DE0030F70AE8F42401F8E9F43400F9E889F075
:1008EE00C2D4F8A9F0227882B60403020980C3E5C7
:1008FE005894014018E54870377805C37994B702CB
:10090E00027812C3E53B9400E53C984020E5486030
:10091E0009855E5D7562FF756301852224E4F53FEE
:10092E00F540F541F542F543F54802098075480159
:10093E00C37994E79402601BE523F43333F913F87B
:10094E00E9540104F9E854FEC39440F8E99400F91F
:10095E0002097CE523F433333333F913F8E95407F2
:10096E000404F9E854F8C39440F8E99400F9883F78
:10097E00894022E548603BC3E53C13F9E53B13F89B
:10098E00C3E53F98F8E54099F9500CC3E89480E927
:10099E0094FF40160209BCC3E8947FE9940050030B
:1009AE000209BC787F79000209BC788079FF8844FF
:1009BE00894522E5486058E5442541F8E54535422C
:1009CE00F9854520E4300701F43543FA30E709C3D1
:1009DE00EA94F040150209FEC3EA940F500302098F
:1009EE00FE78FF79FF7A0F0209FE780079007AF01F
:1009FE00C3E524955C5006E52460094117E54520C2
:100A0E00E70D4117E54530E706884189428A4322C2
:100A1E00E5487003020A81789EE6FAC3E54433F88E
:100A2E00E54533F9119DE930E70BC3E89480E9946D
:100A3E00FF40134158C3E8947FE994005002415897
:100A4E00787F79004158788079FFE820E715C3E573
:100A5E002398F84009C3E894014003020A7F780105
:100A6E00020A7FE8F424012523F84003020A7F7866
:100A7E00FF884622E5487003020AE3789FE6FAA84B
:100A8E0042A943119DE930E70CC3E89401E994FFB4
:100A9E004016020ABAC3E894FFE994005003020A12
:100AAE00BA78FF7900020ABA780179FFE920E715D2
:100ABE00C3E54698F84009C3E894014003020AE1F1
:100ACE007800020AE1E8F424012546F84003020A00
:100ADE00E178FF8824227883E6F52012102075E84D
:100AEE0090E5E820ECF0A8BDA9BE1210B5756855CA
:100AFE00756900C3740013FD745513FC74552CFCFA
:100B0E0074003DFDECFAEDFBC3E89AE99B4014E559
:100B1E00682455F568E5693400F569EA2CFAEB3D71
:100B2E00FB80E5AE68AF69C3E56913F9E56813F8B4
:100B3E00C3E913F9E813F8E56828F566E56939F5B0
:100B4E00677A03C3E913F9E813F8DAF7AA201A70E3
:100B5E0009756800756900020B781AEA6008EE28BC
:100B6E00FEEF39FFDAF88E688F692275E8902278E9
:100B7E0083E6FFE5E820ECF7A8BDA9BE056AC3E54C
:100B8E006A94084052756A00E97007E56B601B02B3
:100B9E000BACC3E8956B6010E56B5006600C14024D
:100BAE000BB80460F9020BB8E56BF56BC394A8F8AB
:100BBE004021755CC0C3E89405F84017755C80C38E
:100BCE00E89405F8400D755C40C3E89405F84003C1
:100BDE00755C0075BB0622EFC39401601BC3E894DD
:100BEE00FFE994035012C3E89568E995695009E549
:100BFE005C600C155C020C0DE55CF46002055CA8F3
:100C0E005CC3E524985002A8248825C3E525955D8C
:100C1E00400B855D25E55DF46003855D5CC3E56A8B
:100C2E00B4070375BB1E223061027832306202783F
:100C3E0050E52C5406601FE879A187F0A4C5F0A2F8
:100C4E00F733F8C3E8955C4002A85C8822882488B4
:100C5E0025306102885E22788FE6FFC3EF9405503F
:0F0C6E0018C3EF94045020C3EF94035028C3EF32
:100C7D0094025030C3EF940150387533A075340F82
:100C8D0075353C75360581CD7533C07534127535A6
:100C9D004075360681CD7533707534177535D07541
:100CAD00360781CD75334C75341D7535C4753609D0
:100CBD0081CD7533287534237535B875360B81CDD7
:100CCD0085334F853450753B00753C0822A84FA9DC
:100CDD0050020CE5A849A94A759100C3E498F59412
:100CED00E499F595759104D25875C820A8CCA9CD75
:100CFD0075C824AA39AB3A8839893AC3E89AF8E914
:100D0D009BF9AA3BAB3CC3EB13FDEA13FCC3ED13FC
:100D1D00FDEC13FCC3EA9CFAEB9DFBEA28FAEB39D8
:100D2D00FB8A3B8B3C400122753BFF753CFF22301B
:100D3D005802A13C759100C3E4954BF594E4954C94
:100D4D00F595759104D258227892E6FF7E10305BAE
:100D5D00027F053063047F037E00A93CA83B7A0423
:100D6D00C3E913F9E813F8DAF7C3E89EF8E994003C
:100D7D00F94009C3E89402E9940050047802E4F9BB
:100D8D00E9FBE8FAC3E913FDE813FCC3EF94036034
:100D9D002EEF20E00DE82CF8E93DF9ECFAEDFB0221
:100DAD000DB9E828F8E939F97A02E4FBC3EF9403A9
:100DBD00400D8A4D8B4E8849894A8C4B8D4C22882B
:100DCD004D894E8A498B4A8C4B8D4C22305802A14D
:100DDD00D9759100C3E4953BF594E4953CF5957573
:100DED009104D25822753E00752000020E01753E09
:100DFD0000752040D2AF053E20580122759D00E5BB
:100E0D003CC313C313F8086030306A06C313C31311
:100E1D00F808C3E8940A4002780A306D08C3E894D4
:100E2D000440027804C3E53C9408400D759D02C34F
:100E3D00E53C94104003759D03205803D2AF2279F1
:100E4D001E206D02790AD2AF0000C2AF205A0A7976
:100E5D003C206D027914306FE03063027978C3E580
:100E6D008B9920630240F740D0E59BF45440B520A8
:100E7D0002C101D8C4D2AF22C25B789CE6146007D0
:100E8D00E53E147002D25B30630B053820581075A7
:100E9D003800020EAC20580715811581021810225A
:100EAD00759100C3E4954DF594E4954EF5957591C6
:100EBD0004D25822AE25305B4F78A3E6FFBF010B5D
:100ECD00D25C752500C2B1C287C281B141305C03CD
:100EDD00752500305802C1DABF020BD25C752500B2
:100EED00C2B1C287C28178A2B6010DB141305C0397
:100EFD00752500305802C1FABF030BD25C75250071
:100F0D00C2B1C287C281D1AD305C037525003058A6
:100F1D0002E115305B04C25C8E2522C2AFC2862071
:100F2D006A03020F4790034B306E0F207502C2808B
:100F3D00307502C2827406D5E0FD207502D2823072
:100F4D007502D280759F02753D02D2AF22C2AF20CD
:100F5D006A03020F7C900302306E17C28620750261
:100F6D00C280307502C2827406D5E0FD020F7F90FB
:100F7D0001E5207502C281307502C2B1305A06E515
:100F8D00256002D287207503759F03307503759F09
:100F9D0001753D03D2AF22C2AF207502C2823075FA
:100FAD0002C280206A03020FC39002C1306E07C2D5
:100FBD00867406D5E0FD207502D280307502D2828E
:100FCD00207503759F01307503759F03753D04D220
:100FDD00AF22C2AF206A03021001900280306E175B
:100FED00207502C282307502C280C2867406D5E0B9
:100FFD00FD0210049001D3C287305A0EE525600A18
:10100D00207502D2B1307502D281759F02753D05F2
:10101D00D2AF22C2AF207502C280307502C28220CB
:10102D006A03021047900237306E0F207502C2829C
:10103D00307502C2807406D5E0FDD2862075037529
:10104D009F03307503759F01753D06D2AF22C2AF68
:10105D00206A030210859003A4306E1F207502C212
:0E106D0082307502C280207502C2803075028A
:10107B00C2827406D5E0FD0210889001F72075023C
:10108B00C2B1307502C281305A0EE525600A207557
:10109B0002D281307502D2B1207503759F01307574
:1010AB0003759F03753D01D2AF229001D1C2B1C22E
:1010BB0087C281C282C286C28022C3E54F9535E5C5
:1010CB005095365001227890E6FFC3EF94055018E7
:1010DB00C3EF9404501BC3EF9403501EC3EF940251
:1010EB005021C3EF94015024C3E54F943CF80211F7
:1010FB0020C3E54F9428F8021120C3E54F941AF84A
:10110B00021120C3E54F9412F8021120C3E54F944E
:10111B000AF8021120E5509400F9884F89502230CB
:10112B00580302112A227880760778817607788215
:10113B007601789476017883760478867609788FB1
:10114B007603789076017895760278927603789B81
:10115B00760D7893760178877602789C760178887D
:10116B0076017889760178857600788C7601788D92
:10117B007600788E76B478967625789776D07898B0
:10118B007678789976C8789A7604789D7600227866
:10119B0093E6FF756409756501C3BF0209756405A4
:1011AB007565010211DFC3BF03097564057565021F
:1011BB000211DFC3BF04097564057565030211DFF6
:1011CB00C3BF0506756409756507C3BF060675645D
:1011DB00007565007887E6FFC26CC3BF0302D26C53
:1011EB00C26BC26A7418552D6002D26AC26E60025D
:1011FB00D26ED26F6002C26FC2757888E630E102A0
:10120B00D275C2767889E630E102D276C3EF9402CA
:10121B006008758E01D26D02122A758E00C26D2286
:10122B007880E61490008093789EF67881E614908F
:10123B00008093789FF611B522789BE61490008D71
:10124B009378A0F611B5227886E61490009A9378DD
:10125B00A1F611B522789CE6149000A79378A2F61C
:10126B00789CE6149000AC9378A3F611B522C2B328
:10127B00789DE66002D2B3227896E6FA7897E6FB81
:10128B003077047A007BFFC3EB9AFCC39482500245
:10129B007C82756C00056CEC856CF0A4C3E5F09456
:1012AB008040F222C2D353D9BF7581C043FF801255
:1012BB0007D275EF0243B203E5B324044002F5B342
:1012CB0075803875A4C775F1FF75D4DF7590FF7500
:1012DB00A50075F20075D50075A0FF75A60075F316
:1012EB000075D60075B0E475A71B75F4FF75E24168
:1012FB0011B5E4F8F6D8FD313112185D319A512B46
:10130B00514451525160517951837898866D11B582
:10131B0075885075890275C82475910475D840126B
:10132B0007E61207F51207DE1207FC1207DE12089A
:10133B00031207DE121CE51207E61207E61207E29C
:10134B0075A82275B80275E69075F610759B8075B9
:10135B009D0375D10E75BC5875BB0675BA1F75E824
:10136B00801207D2D2AF120AE443DA01C2D8C269A3
:10137B001207E6753001D2597A05E55770027A05E6
:10138B001207D6E558C3940240EEE52E541F855A3A
:10139B0059F55AB559E2DAE2C25953DACF2076033E
:1013AB0043DA2030760343DA10C2D8C2691207E25F
:1013BB001207D67802741F552E70027800C3E558B9
:1013CB009840EDC2AF1207F51207F51207F5D2AF31
:1013DB001207E67547001207D6788CE6C3940150C6
:1013EB00030214AAE530C3940150030214AA741F1C
:1013FB00552E6035C3E55894FF50030214AAC2AFB3
:10140B0012080AD2AF1207E2C3E558940150EFC29B
:10141B00AF1207F51207DA1207F5D2AF1207E2C3C4
:10142B00E55894FF40E9021D6A7F05D2775183127C
:10143B0007E2C2AFC2775183C3E558947FD2AF4066
:10144B0068C2AF12080AD2AFDFE1C3E55894057842
:10145B0097F61207E612190D121CED7F0AD277517F
:0F146B00831207E2C2AFC2775183C3E558947F63
:10147A00D2AF50E8C2AF1207F51207DA1207F5D257
:10148A00AFDFDBE55824057896F61207E612190D48
:10149A00121D1C1207E2C3E55894FF40F6021D6AAA
:1014AA00C3E558954740038558471207E2C3E558F4
:1014BA009401400261E1C2AF12080A12080A120836
:1014CA000AD2AF1207E6753000E4F531F53205317C
:1014DA00E531F470360532789AE678281460127885
:1014EA005014600D78A014600878F0146003753207
:1014FA0000C3E53298401415327899866DC2AF124E
:10150A00080AD2AF7898866D1207E21207D6E52844
:10151A007008741F552E70026181C3E55894064005
:10152A00AD1207E2E528700302138111B5E4F52232
:10153A00F523F524F525755CFF7885865FF53FF57B
:10154A0040F541F542F543F56AF548F52BF52CF5DA
:10155A005B120C65756A0875BB1E1207D2120B79ED
:10156A00E5E820ECFBA8BDA9BEE97001F8886B127A
:10157A000B7D756A0875BB1E7895E630E003021587
:10158A00C57887E6FE7602319A7887EEF6D261C28E
:10159A00AF120C3585225C85225DD2AFC2617525FA
:1015AA0000756200756301D260D26375380011203C
:1015BA00115B120CE1120C650216E77887E6FE76DB
:1015CA00037893E6FD7605319A7887EEF67893EDFF
:1015DA00F6D260D261D26E1120115B120C3512075D
:1015EA00D2120F281207D21207D2120F5A1207D696
:1015FA00120FA41207D61207D6120FDF1207DA113A
:10160A00201207D61207D2C261D262120B79120BCC
:10161A007D120C35756A0875BB1E115B120CDA1245
:10162A000D5511C5312A120F28120CDA120D551157
:10163A00C5312A120F5A120CDA120D5511C5312A68
:10164A00120FA4120CDA120D5511C5312A120FDF2E
:10165A00120CDA120D5511C5312A1120120CDA12A8
:10166A000D5511C5C3E54F9535E5509536400C31FA
:10167A002AC3E55894015093021810312AC262789D
:10168A0087E6FE7602319A7887EEF685225C855ED9
:10169A005D855E25756200756301D263753800C287
:1016AA00AF207502C282307502C280207502C280E4
:1016BA00307502C282742DD5E0FDD2AF115B120CD7
:1016CA00E1120D3C120D55120DD9756A0075BB0653
:1016DA000216E7319A115B756A0075BB06120DFB9B
:1016EA00120E85120EAD1208F4120EC1120F281234
:1016FA000CE1120D3C120D55120DD9120DF2120EFB
:10170A0085120EAD120981120EC1120F5A120CE186
:10171A00120D3C120D55120DD9120DFB120E851227
:10172A000EAD1209C1120EC1120FA4120CE1120D54
:10173A003C120D55120DD9120DF2120E85120EAD74
:10174A00120A1E120EC1120FDF120CE1120D3C1208
:10175A000D55120DD9120DFB120E85120EAD120A7D
:10176A0082120EC11120120CE1120D3C120D5512FB
:10177A000DD9120DF2120B79120E85120EAD120B43
:10178A007D120EC1115B120CE1120D3C120D5512A5
:10179A000DD930632A855E5C855E5D75620075636E
:1017AA0001C3E5389464400AC263D26475371402EF
:1017BA0017C9C3E558940140030216E7021810300E
:1017CA006419E537147005C2640216DDF537C3E5FE
:1017DA0058940140030216E7021810C3E55B94010E
:1017EA004009855E5D7562FF756301C3E55B94FA26
:1017FA005014741F552E7004E528600AC3E53C9402
:10180A00F050030216E71210B57887E6FE76021248
:10181A00119A7887EEF6E4F522F523F524F525F5F5
:10182A005FC2601207D21210B5741F552E7007E5F9
:10183A002870030213817895E630E009121CE5123C
:10184A001CE5121CE5788DE6C3940140030213BB24
:10185A000214D3901A0D7820121C00E520B4A50CAE
:0F186A00A3121C00E520B45A0302187F1211319B
:1018790012190D02190C901A037880121C00A30882
:10188900121C00A308121C00A308121C00A308A321
:1018990008A308121C00A308121C00A308121C00AC
:1018A900A308121C00A308A308A308121C00A3087C
:1018B900121C00A308121C00A308121C00A3081282
:1018C9001C00A308A308121C00A308121C00A308EB
:1018D900121C00A308121C00A308121C00A3081262
:1018E9001C00A308121C00A308121C00A308121C48
:1018F90000A308121C00A308121C00A308121C0054
:10190900901A2122C2AF121C3F121C19901A00749E
:101919000A121C05A37404121C05A37410121C05D9
:10192900901A037880121C04A308121C04A308123D
:101939001C04A308121C04A308A308A308121C046E
:10194900A308121C04A308121C04A308121C04A354
:1019590008A308A308121C04A308121C04A3081254
:101969001C04A308121C04A308121C04A308A3083E
:10197900121C04A308121C04A308121C04A30812B5
:101989001C04A308121C04A308121C04A308121C9B
:1019990004A308121C04A308121C04A308121C04A3
:1019A900A308121C04A308121C04121C52121C3096
:0419B900901A21223D
:101A00000A041007070104FFFF09020101A55A019A
:101A100000B40301FF0301010225D078C8040D01C1
:021A200000FFC5
:101A4000235475726E6967794145343541232020EE
:101A500023424C48454C4923463331302320202033
:101A60002020202020202020202020202020202076
:101C0000E493F622E6438F01538FFD75EF0275B71B
:101C1000A575B7F1F0538FFE22438F02438F0175F4
:101C2000EF0275B7A575B7F1901A0DF0538FFC222E
:101C3000901A0D74A59105901A0E745A9105227A86
:101C40003079D07820901A409100E520F709A3DA86
:101C5000F7227A3079D0901A40E7910509A3DAF992
:101C600022AB6EA86FBB01057980021CE2BB0205A6
:101C70007981021CE2BB03057982021CE2BB0405E8
:101C80007994021CE2BB05057983021CE2BB0605C0
:101C90007995021CE2BB07057986021CE2BB0805A8
:101CA000798F021CE2BB09057990021CE2BB0A0590
:101CB0007992021CE2BB0B05799B021CE2BB0C056E
:101CC0007993021CE2BB0D057987021CE2BB0E056D
:101CD000799C021CE2BB0F057988021CE27989021B
:101CE0001CE2E8F7227C051207E6DCFB22C2AF12F9
:101CF00007F51207FC12080312080A1207DA120786
:101D0000F51207FC12080312080A1207DA1207F587
:101D10001207FC12080312080AD2AF22C2AF12083F
:101D20000A1208031207FC1207F51207DA12080A52
:101D30001208031207FC1207F51207DA12080A123A
:101D400008031207FC1207F5D2AF22AE6EAF6FC2C6
:101D5000AF1207F51207F51207F51207DADEF212D5
:101D6000080A1207DADFF8D2AF2291ED91E591E58A
:101D7000756E01756F01757000B14B7C05AD581221
:101D800007E6C3ED955870F5C3E55894014009C3C3
:101D9000E55894FF4032A1A6916112190D91EDC250
:101DA000AF75EF1291E5DCD50570C3E57094035073
:101DB0000280C691E5056FE56E149000B193F808B6
:101DC000C3E56F98500280AE91E591E5056EC3E5DD
:101DD0006E94115002809C12113112190DC2AF7510
:041DE000EF1291E588
:00000001FF
